:100000000C9467080C948F080C948F080C948F083C
:100010000C948F080C948F080C948F080C948F0804
:100020000C948F080C948F080C948F080C948F08F4
:100030000C948F080C948F080C948F080C948F08E4
:100040000C941B280C948F080C948F080C948F0828
:100050000C948F080C948F080C948F080C948F08C4
:100060000C94521B0C948F0820202020202020204C
:100070004241434B202000202020202020205343B9
:100080004F5045200020205345542046494C5445AC
:1000900052204C204D20480020202020202020539A
:1000A00045415243482000202020202020202000CD
:1000B0000000000000000000000000000000000040
:1000C00000000000007800000000000000F80000C0
:1000D0000000000000F800000000000001F800002F
:1000E0000000000071F0000000000000F1F3E000EB
:1000F00000000001F1F3E00000000001F1F3E00076
:1001000000000003F1E3E00000000003F3E3E0007F
:1001100000000001F3E3E00000000001C3E3E000A1
:1001200000000003E3E3E00000000003E3E3C0009D
:1001300000000003E3C3E00000000003E383E1E00C
:1001400000000003E383E3F000000001C383E3F851
:100150000000000107C3C3F80000000387C3C3F811
:1001600000000007C7C383F00000000787C7C3F083
:100170000000000F87C7C1F00000000F87CFC0F05C
:100180000000000F838FC3F000000007800FC3F052
:1001900000000001000783F000000000000303E0FE
:1001A00000000003800003E010000007E60007C025
:1001B0003C00000FFFF80FC07E00000FFFFC0FC0D7
:1001C0003F80000FFFFE0FC01FC0000FFFFFC78062
:1001D0000FC0000FBFDFF70007C0000F7FEFFC006C
:1001E00003C0000F7FEFFE00000000067FE7FE0067
:1001F000000000027FE7FE000000000730EFFF0074
:100200000000003F060FFF00000000FF0F0FFF007F
:10021000000003FC0003FF00000007F00F00FF00D8
:1002200000000FC00F063F0000001FDE4FA79F0019
:1002300000001FBF7F6FDF0000003FBF204FFF00A7
:1002400000003FBF905FFE0000007FFFC03FFC004A
:1002500000007FFFE07FF80000003FFFE63FF00076
:1002600000003FFFCF1FE00000001FFE3FC1C000A5
:1002700000000FFFFFFF8000000003FFFFFF0000F2
:10028000000000FFFFFE00000000007FFFFC0000F8
:100290000000003FFFF800000000000FFFF000002A
:1002A00000000003FC00000000000000000000004F
:1002B000000000000000000000000000000000003E
:1002C000000000000000000000000000000000002E
:1002D000000000030000000000000003FFFFF0002A
:1002E00000000003B00000000000000180000000DA
:1002F00000000003C000000000000003C000000078
:1003000000000003C000000000000003C000000067
:1003100000000003C000000000000003C000000057
:1003200000000003C000000000000003C000000047
:1003300000000003C000000000000007C000000033
:10034000000003FFFFC00000000003FFFFC000002B
:100350000000020FE04000000000027FFC400000AF
:100360000000027FFE4020000004027FFE402000CB
:10037000000007FFFFC000000007FFBFFFFFE00015
:100380000007FFFFFBFFE000000F3DFFF7BDF0009F
:10039000000F18FFFF18F000001F18FFFF18F000F3
:1003A000001FBDFFFFBDF800001FFFFFFFFFF800AB
:1003B000001F83FFFFC3F800001F38FEFF18F8007E
:1003C000001EFE7D7E7E7800001DFF7E7CFF3800D3
:1003D000001D01AFED00B800001911A7ED01B80034
:1003E000001BFFBFFDFFB800001911A7ED99B80071
:1003F000001901A7ED00B800001DFF7C3CFF38008C
:10040000001EFE7DBE7E7800001F38FDBF3CF80058
:10041000001F83FDFF81F800001FFFFC7FFFF80035
:10042000001FD3FC7FDBF800001FDFFFFFDBF800BD
:10043000001FFFFFFFFFF800001FFF8021FFF800F3
:10044000001F9F0001F9F800001F1F0001F8F000D5
:10045000001F370001E8F000000F230001CCF0007E
:10046000000F230001C5F000000FFF0001FFE000B6
:100470000007FF0001FFE0000003FFBFFDFFC00019
:100480000001FFFFFFFF000000001DFFFF20000034
:10049000000000000000000000000000000000005C
:1004A000000000000000000000000000000000004C
:1004B000000000000000000000000000000000003C
:1004C000000000000000000000000000000000002C
:1004D000000000000000000000000000000000001C
:1004E000000080000000000000010000000000008B
:1004F00000010000000000000003000000000000F8
:1005000000030000000040000003800000004000E5
:100510000003C0000000C0000007C0380001C00098
:100520000007C0780601C0000007C3FE3F81C0007D
:100530000007CFFFFFF1C0000007FFFE3FF9C0003A
:100540000007FFFC3FFFC0000007FFF81FFFC000CF
:1005500000079FF89FFFC00000039FFBEFFCC00057
:1005600000039FF7EFF8C00000038FEFF7F8C0001B
:10057000000387CFF3F0C0000003801FF800C00025
:100580000003833FFC00C0000003C3FFFF80C000E6
:100590000001E3FFFFC1C0000001FFFFFFF7800083
:1005A0000001FFF7EFFF80000001FFEFF7FF800081
:1005B0000018FFEFF7FF9000007CFFE427FF3E00EC
:1005C00001FEFFE3C7FF7F8007FF7F8001FEFFE0A2
:1005D0003FFFFF399CFCFFFC7FFFFF65A6FFFFFE8E
:1005E0007FFFFFF66FFFFFFE3FFFFFF24FFFFFFCB5
:1005F0001FFFFFFA5FFFFFF81FFF3FFE7FFCFFF8C2
:100600001FF07FFC3FFE0FF81F30FFE387FF0CF861
:100610000611FFFFFFFF88E00719F87FFE7F90E0DB
:10062000071FFC3FFC3FF9E003BFFC3FF83FFDC064
:1006300001FFFC1FF83FFF8001FFFE7FFE7FFF8070
:1006400000FFFEFFFE7FFF00003FFE3FFC7FFC003F
:10065000003FFC3FFC3FFC00001FF03FF80FFC0098
:10066000003FC0181803F800001F00000000FC0045
:10067000001C000000003800000800000000180006
:10068000000000000000000000000000000000006A
:10069000000000000000000000000000000000005A
:1006A000000000000000000000000000000000004A
:1006B000FFFFFFFFFFFFFFFFFFFFFFFFFFFFFFFF4A
:1006C000F7FFFFEFFF7FBF7BDEFDFEFFF7FFFFEFD2
:1006D000F8F9F9F3F73F3F719CF8FCCFCF9F9F1FCC
:1006E000FC1C7C71F11F1F218CB8F88F8E3E383FA7
:1006F000E6000C38700E06000810701E18380067EF
:10070000F000000818020200000060181060001FCE
:10071000FC00000000000000000000000000003F9E
:10072000FF0000000000000000000000000000FFCB
:10073000F1C000000000000000000000000003CF36
:10074000FC00000000000000000000000000003F6E
:10075000FF0000000000000000000000000000FF9B
:10076000FFC000000000000000000000000003FFC8
:10077000F1F00000000000000000000000000F8FFA
:10078000FC08000000000000000000000000303FF6
:10079000FF0000000000000000000000000000FF5B
:1007A000FFC000000000000000000000000007FF84
:1007B000F80000000000000000000000000000073A
:1007C000FFC0000000000000000000000000003F2B
:1007D000FFFC00000000000000000000000000FF1F
:1007E000E00000000000000000000000000003FF27
:1007F000FC00000000000000000000000000007F7E
:10080000FFC00000000000000000000000003FFFEB
:10081000FFFC000000000000000000000000000FCE
:10082000FF0000000000000000000000000007FFC3
:10083000FE00000000000000000000000000003F7B
:10084000F000000000000000000000000000003F79
:10085000FF8000000000000000000000000000FF1A
:10086000FF00000000000000000000000000001F6A
:10087000FF800000000000000000000000000FFFEB
:10088000FC00000000000000000000000000000F5D
:10089000FF00000000000000000000000000007FDA
:1008A000F000000000000000000000000000000751
:1008B000FFF800000000000000000000000007FF3B
:1008C000FFF0000000000000000000000003FFFF38
:1008D000F80000000000000000000000000001FF20
:1008E000FFF0000000000000000000000000003FDA
:1008F000FF00000000000000000000000000001FDA
:10090000FE00000000000000000000000000007F6A
:10091000F000000000000000000000000000000FD8
:10092000C3000000000000000000000000001FC322
:10093000FF8000000000000000000000000003FF36
:10094000FFF0000000000000000000000000000FA9
:10095000FF8000000000000000000000000007FF12
:10096000FF0000000000000000000000000000FF89
:10097000FF00000000000000000000000000000F69
:10098000FF000000000000000000000000000FFF5A
:10099000FC0000000000000000000000000001FF5B
:1009A000FFF0000000000000000000000000007FD9
:1009B000FFC0000000000000000000000000000F69
:1009C000FF00000000000000000000000000007FA9
:1009D000FC00000000000000000000000000303FAC
:1009E000F1F00000000000000000000000000F8F88
:1009F000FFC000000000000000000000000003FF36
:100A0000FF0000000000000000000000000000FFE8
:100A1000FC00000000000000000000000000003F9B
:100A2000F000000000000000000000000000038F44
:100A3000FF0000000000000000000000000000FFB8
:100A4000FC00000000040000000020000000003F47
:100A5000F8000600180E0800001070001000001FBB
:100A6000E6001C00701E08100810780018000067CF
:100A7000FC1C7C01F11F1C318C38F88C0E36383F81
:100A8000F8F9F873F3BF3C799C38FDCF8F9F9F1F17
:100A9000F7FFFFEFFFFFBD7BDEBDFFFFF7FFFFEFBF
:100AA000FFFFFFFFFFFFFFFFFFFFFFFFFFFFFFFF56
:100AB000E916D516C116AD169916851671165D166E
:100AC000651678168B169E16B116C416D716EA163A
:100AD0004916351621160D16FD161117251739174B
:100AE0006C1680169416A816BC16D016E416F816C6
:100AF0001A163F1664168916AE16D316F8161D1769
:100B0000F21417153C1561158615AB15D015F515A2
:100B1000052A9B29912987291D29132909299F28FD
:100B200003290C2916291F29892992299C29052A7C
:100B300095288B28812817280F2A192A832A8D2A7D
:100B4000062910291A2984298E299829022A0C2A73
:100B50001D288F2802291429872999290C2A1E2A41
:100B600009261C268E2601271327862798270B285F
:100B700000000000003E5B4F5B3E3E6B4F6B3E1C37
:100B80003E7C3E1C183C7E3C181C577D571C1C5E4E
:100B90007F5E1C00183C1800FFE7C3E7FF00182425
:100BA0001800FFE7DBE7FF30483A060E26297929CF
:100BB00026407F050507407F05253F5A3CE73C5A04
:100BC0007F3E1C1C08081C1C3E7F14227F22145FE1
:100BD0005F005F5F06097F017F006689956A60603C
:100BE00060606094A2FFA29408047E040810207E36
:100BF000201008082A1C08081C2A08081E101010BB
:100C0000100C1E0C1E0C30383E3830060E3E0E0600
:100C1000000000000000005F000000070007001453
:100C20007F147F14242A7F2A122313086462364912
:100C30005620500008070300001C224100004122FA
:100C40001C002A1C7F1C2A08083E080800807030FF
:100C5000000808080808000060600020100804026E
:100C60003E5149453E00427F400072494949462174
:100C700041494D331814127F1027454545393C4AE8
:100C800049493141211109073649494936464949FF
:100C9000291E000014000000403400000008142247
:100CA00041141414141400412214080201590906B5
:100CB0003E415D594E7C1211127C7F494949363EB6
:100CC000414141227F4141413E7F494949417F099C
:100CD0000909013E414151737F0808087F00417FA7
:100CE00041002040413F017F081422417F404040A5
:100CF000407F021C027F7F0408107F3E4141413E3D
:100D00007F090909063E4151215E7F0919294626BE
:100D10004949493203017F01033F4040403F1F20C2
:100D200040201F3F4038403F631408146303047899
:100D300004036159494D43007F41414102040810B9
:100D400020004141417F04020102044040404040F4
:100D5000000307080020545478407F284444383862
:100D600044444428384444287F38545454180008D4
:100D70007E090218A4A49C787F0804047800447DAE
:100D800040002040403D007F1028440000417F404B
:100D9000007C047804787C0804047838444444389F
:100DA000FC1824241818242418FC7C08040408487F
:100DB0005454542404043F44243C4040207C1C20D0
:100DC00040201C3C4030403C44281028444C90902B
:100DD000907C4464544C4400083641000000770085
:100DE00000004136080002010204023C2623263C92
:100DF0001EA1A161123A4040207A3854545559211D
:100E00005555794122545478422155547840205404
:100E10005579400C1E527212395555555939545452
:100E2000545939555454580000457C410002457DC1
:100E3000420001457C407D1211127DF0282528F0EA
:100E40007C545545002054547C547C0A097F493217
:100E5000494949323A4444443A324A4848303A418E
:100E600041217A3A42402078009DA0A07D3D424237
:100E7000423D3D4040403D3C24FF2424487E4943C0
:100E8000662B2FFC2F2BFF0929F620C0887E090333
:100E900020545479410000447D413048484A32385A
:100EA0004040227A007A0A0A727D0D19317D262986
:100EB000292F28262929292630484D40203808087E
:100EC000080808080808382F10C8ACBA2F102834B2
:100ED000FA00007B000008142A142222142A1408A5
:100EE0005500550055AA55AA55AAFF55FF55FF00B4
:100EF0000000FF00101010FF00141414FF00101069
:100F0000FF00FF1010F010F0141414FC001414F77C
:100F100000FF0000FF00FF1414F404FC1414171069
:100F20001F10101F101F1414141F00101010F000B9
:100F30000000001F101010101F10101010F01000F3
:100F40000000FF101010101010101010FF10000003
:100F500000FF140000FF00FF00001F10170000FC3E
:100F600004F414141710171414F404F40000FF0010
:100F7000F714141414141414F700F7141414171499
:100F800010101F101F141414F4141010F010F0009F
:100F9000001F101F0000001F14000000FC140000C0
:100FA000F010F01010FF10FF141414FF14101010A4
:100FB0001F00000000F010FFFFFFFFFFF0F0F0F057
:100FC000F0FFFFFF0000000000FFFF0F0F0F0F0FEB
:100FD0003844443844FC4A4A4A347E020206060237
:100FE0007E027E0263554941633844443C04407E9E
:100FF000201E2006027E020299A5E7A5991C2A4917
:101000002A1C4C7201724C304A4D4D3030487848A1
:1010100030BC625A463D3E494949007E0101017E8D
:101020002A2A2A2A2A44445F444440514A444040E0
:10103000444A51400000FF0103E080FF000008081F
:101040006B6B083612362436060F090F060000189F
:10105000180000001010003040FF0101001F0101C6
:101060001E00191D1712003C3C3C3C000000000013
:101070000000000800020100000304070000000057
:101080000000000001020408102040800102040852
:1010900010200102040810200404040404040404C1
:1010A0000202020202020303030303030000000022
:1010B00023002600290000000000250028002B0046
:1010C00000000000240027002A00E819B01A1124AB
:1010D0001FBECFEFD8E0DEBFCDBF16E0A0E0B1E08D
:1010E000E8EAFDE502C005900D92AC39B107D9F7E9
:1010F00027E0ACE9B6E001C01D92A53DB207E1F7DB
:1011000010E1CEECD0E104C02297FE010E94A42E93
:10111000CA3CD107C9F70E94172C0C94D22E0C940C
:1011200000000C94BC2E0C94C42EACE9B6E020E078
:10113000FC013491332331F02E3121F03D9301969F
:101140002F5FF6CFE22FF0E0E456F94F30838CE9C1
:1011500096E0089560E08FE00E94872981E090E0AA
:101160000E94C22861E081E10E94872981E090E02D
:101170000E94C22861E08FE00E94872981E090E010
:101180000E94C22860E08FE00E94872981E090E001
:101190000C94C22860E08FE00E94872981E090E0F3
:1011A0000E94C22860E081E10E94872981E090E0EE
:1011B0000E94C22861E08FE00E94872981E090E0D0
:1011C0000E94C22860E08FE00E94872981E090E0C1
:1011D0000C94C22881E090E00E94C22860E080E187
:1011E0000E94872981E090E00C94C22881E090E081
:1011F0000E94C22861E080E10E94872981E090E09E
:101200000C94C2281F93CF93DF9360910A0160333F
:1012100019F4E091C60626C0613319F4E091C506C1
:1012200021C0623319F4E091C4061CC0633319F481
:10123000E091C30617C0643319F4E091C20612C0EE
:10124000653319F4E091C1060DC0663319F4E091DD
:10125000C00608C0673319F4E091BF0603C06033CD
:1012600040F4E62FF0E0EE0FFF1FE05FF44FC59172
:10127000D49181E090E00E9493080E94F60881E0FA
:1012800090E00E94C2280E94EA080E94CA080E94B8
:10129000CA080E94CA080E94AA080E94CA0814E14B
:1012A0000E94CA081150E1F70E94F60862E070E05F
:1012B00080E090E00E94882881E090E00E94C228AF
:1012C0000E94EA080E94F6080E94EA080E94AA0802
:1012D0000E94CA080E94CA080E94CA080E94AA085E
:1012E00010E1C0FF03C00E94AA0802C00E94CA0801
:1012F000D695C7951150A9F70E94CA080E94CA083E
:101300000E94CA080E94CA080E94F60881E090E084
:101310000E94C22860E080E10E94872960E08FE09F
:101320000E94872960E081E1DF91CF911F910C94A9
:1013300087298F929F92AF92BF92CF92DF92EF92C6
:10134000FF928091CB069091CC0601969093CC06AB
:101350008093CB068091C9069091CA06019690931E
:10136000CA068093C90684E10E940829BC01882727
:1013700077FD8095982F0E942B2D60930407709322
:101380000507809306079093070769E170E080E006
:1013900090E00E94882885E10E940829BC018827E6
:1013A00077FD8095982F0E942B2D6B017C01609317
:1013B00000077093010780930207909303078090C2
:1013C000040790900507A0900607B09007072091AA
:1013D00018013091190140911A0150911B01C5016A
:1013E000B4010E94DB2D181644F4809218019092EB
:1013F0001901A0921A01B0921B01209110013091A5
:1014000011014091120150911301C701B6010E94D0
:10141000DB2D181644F4C0921001D0921101E09215
:101420001201F092130120911C0130911D01409195
:101430001E0150911F01C501B4010E948C2C87FF31
:1014400008C080921C0190921D01A0921E01B092D2
:101450001F01209114013091150140911601509106
:101460001701C701B6010E948C2C87FF08C0C092EB
:101470001401D0921501E0921601F0921701A70114
:101480009601C501B4010E94DB2D181624F41092B8
:10149000CA061092C906A7019601C501B4010E94AF
:1014A0008C2C87FF04C01092CC061092CB06809142
:1014B000200190E02091CB063091CC068217930753
:1014C00018F41092CD060AC02091C9063091CA06C0
:1014D0008217930718F481E08093CD068091CD06A2
:1014E00081113BC060E085E00E9487296091210165
:1014F00070E080E090E00E94882861E086E00E9431
:10150000872960E08DE00E94872948E250E068E486
:1015100070E081ED96E00E944E2280910C018823BC
:10152000C1F080910E018430A1F463E375E081ED98
:1015300096E00E94242A4AE350E06BE470E081EDDB
:1015400096E00E944E226BE375E081ED96E00E94EA
:10155000242A81ED96E00E945E278091CD0681309D
:1015600009F043C060E086E00E9487296091210174
:1015700070E080E090E00E94882861E085E00E94B1
:10158000872961E08DE00E94872948E250E068E405
:1015900070E081ED96E00E944E2280910C0188233C
:1015A000C1F080910E018430A1F460E475E081ED1A
:1015B00096E00E94242A4AE350E062E670E081ED62
:1015C00096E00E944E2268E475E081ED96E00E946C
:1015D000242A81ED96E0FF90EF90DF90CF90BF90AE
:1015E000AF909F908F900C945E27FF90EF90DF90CC
:1015F000CF90BF90AF909F908F9008954F925F9241
:101600006F927F928F929F92AF92BF92CF92DF9212
:10161000EF92FF920F931F93CF93DF9300D000D0F0
:10162000CDB7DEB784E10E940829BC01882777FD89
:101630008095982F0E942B2D6093040770930507C7
:10164000809306079093070769E170E080E090E0DF
:101650000E94882885E10E940829BC01882777FD1F
:101660008095982F0E942B2D4B015C016093000701
:10167000709301078093020790930307C0900407BB
:10168000D0900507E0900607F09007072091180119
:101690003091190140911A0150911B01C701B60107
:1016A0000E94DB2D181644F4C0921801D092190143
:1016B000E0921A01F0921B0120911001309111016A
:1016C0004091120150911301C501B4010E94DB2D1C
:1016D000181644F48092100190921101A092120108
:1016E000B092130120911C0130911D0140911E0107
:1016F00050911F01C701B6010E948C2C87FF08C0C2
:10170000C0921C01D0921D01E0921E01F0921F01B7
:10171000209114013091150140911601509117014B
:10172000C501B4010E948C2C87FF08C0809214016F
:1017300090921501A0921601B092170160911C01C0
:1017400070911D0180911E0190911F010E94F82C43
:101750002B013C01609118017091190180911A01CF
:1017600090911B010E94F82C9B01AC01C701B601AE
:1017700029833A834B835C830E94F82C1F921F922B
:101780001F9222E0922E9F9232E3A32EB12CC12C05
:10179000D12C8301720129813A814B815C810E94A5
:1017A000CD2B0E942B2D6093040770930507809327
:1017B00006079093070760911401709115018091BD
:1017C0001601909117010E94F82C2B013C016091A9
:1017D00010017091110180911201909113010E94EA
:1017E000F82C9B01AC01609100077091010780917A
:1017F00002079091030729833A834B835C830E94FD
:10180000F82C1F921F921F929F92830172012981CF
:101810003A814B815C810E94CD2B0E942B2D6093DD
:1018200000077093010780930207909303070FB698
:10183000F894DEBF0FBECDBF0F900F900F900F90AA
:10184000DF91CF911F910F91FF90EF90DF90CF909C
:10185000BF90AF909F908F907F906F905F904F90D0
:1018600008958F929F92AF92BF92CF92DF92EF92A4
:10187000FF920F931F93CF93DF9381ED96E00E9429
:10188000AE258AE00E94BD2921E0892B09F420E0E1
:1018900020930D0188E00E94BD2921E0892B09F4E5
:1018A00020E020930C0183E00E94BD2921E0892BD8
:1018B00009F420E020930B0180910C01811110921A
:1018C000BD0680910D01811143C080910A018F5F97
:1018D000873308F087E380930A0181ED96E00E9448
:1018E000AE2564E081ED96E00E94542244E150E090
:1018F00060E070E081ED96E00E944E226DE475E0BC
:1019000081ED96E00E94242A81ED96E00E945E27F8
:1019100068EC70E080E090E00E94882861E081ED52
:1019200096E00E9454220E9402098FE590E0909375
:10193000CF068093CE0681E08093C7061092BB0647
:101940001092BA066AE070E080E090E00E94882879
:1019500080910B01811140C080910A0181508093D8
:101960000A0181ED96E00E94AE2564E081ED96E0EB
:101970000E94542244E150E060E070E081ED96E086
:101980000E944E2265E575E081ED96E00E94242AD2
:1019900081ED96E00E945E2768EC70E080E090E0C8
:1019A0000E94882861E081ED96E00E9454220E9406
:1019B00002098FE590E09093CF068093CE0682E0F7
:1019C0008093C7061092BB061092BA066AE070E0D8
:1019D00080E090E00E94882880910C01811122C251
:1019E0008091BD068F5F8093BD061092C80610924D
:1019F000BB061092BA06C091C806CA3008F5CF5F80
:101A0000C093C80681ED96E00E9467222C2F30E03B
:101A1000220F331F97FD0196AC015595479501E0C4
:101A200010E06FE370E081ED96E00E94271E81EDEB
:101A300096E00E945E2761E08DE00E948729DBCF5F
:101A40008091BD06863010F01092BD068091BD06D3
:101A5000813009F08AC081ED96E00E94AE2562E0F7
:101A600081ED96E00E94542244E150E060E070E095
:101A700081ED96E00E944E226EE575E081ED96E0E4
:101A80000E94242A81ED96E00E945E2768E572E0BC
:101A900080E090E00E94882861E081ED96E00E945D
:101AA000542281ED96E00E94AE2564E670E080E06D
:101AB00090E00E94882888E00E94BD2921E0892BBF
:101AC00009F420E020930C01222309F462C410924F
:101AD000BD0681ED96E00E94AE2562E081ED96E0C4
:101AE0000E94542244E150E060E070E081ED96E015
:101AF0000E944E2267E675E081ED96E00E94242A5E
:101B000081ED96E00E945E2780910A01885F8F3206
:101B100008F08FE280930A010E94020980E590E0BC
:101B20009093CF068093CE0660E471E080E090E071
:101B30000E94882861E081ED96E00E94542281EDA8
:101B400096E00E94AE2560E471E080E090E0DF91D5
:101B5000CF911F910F91FF90EF90DF90CF90BF90AA
:101B6000AF909F908F900C948828823009F078C0B5
:101B700081ED96E00E94AE2562E081ED96E00E9444
:101B8000542244E150E060E070E081ED96E00E9474
:101B90004E226CE675E081ED96E00E94242A81EDEC
:101BA00096E00E945E2768E572E080E090E00E9487
:101BB000882861E081ED96E00E94542281ED96E054
:101BC0000E94AE2588E00E94BD2921E0892B09F4FE
:101BD00020E020930C01222309F4DBC31092BD0600
:101BE00081ED96E00E94AE2562E081ED96E00E94D4
:101BF000542244E150E060E070E081ED96E00E9404
:101C00004E2267E675E081ED96E00E94242A81ED80
:101C100096E00E945E2780910A01885080930A0115
:101C20000E94020980E590E09093CF068093CE0653
:101C300060E471E080E090E00E94882861E081ED3E
:101C400096E00E94542281ED96E00E94AE2560E469
:101C500071E080E090E00E9488281092BC0699C351
:101C6000833009F066C081ED96E00E94AE2562E007
:101C700081ED96E00E94542244E150E060E070E083
:101C800081ED96E00E944E2265E775E081ED96E0D9
:101C90000E94242A81ED96E00E945E2768E572E0AA
:101CA00080E090E00E94882881ED96E00E94AE25B9
:101CB00088E00E94BD2921E0892B09F420E02093CF
:101CC0000C01222309F465C31092BD0681ED96E054
:101CD0000E94AE2562E081ED96E00E94542244E12C
:101CE00050E060E070E081ED96E00E944E2267E6F1
:101CF00075E081ED96E00E94242A81ED96E00E9435
:101D00005E2760E471E080E090E00E94882861E056
:101D100081ED96E00E94542281ED96E00E94AE256E
:101D200060E471E080E090E00E94882885E0809384
:101D30000E018091BD06843009F065C081ED96E00A
:101D40000E94AE2562E081ED96E00E94542244E1BB
:101D500050E060E070E081ED96E00E944E226DE779
:101D600075E081ED96E00E94242A81ED96E00E94C4
:101D70005E2768E572E080E090E00E94882881EDAF
:101D800096E00E94AE2588E00E94BD2921E0892BC3
:101D900009F420E020930C01222309F4FAC21092E6
:101DA000BD0681ED96E00E94AE2562E081ED96E0F1
:101DB0000E94542244E150E060E070E081ED96E042
:101DC0000E944E2267E675E081ED96E00E94242A8B
:101DD00081ED96E00E945E2760E471E080E090E093
:101DE0000E94882861E081ED96E00E94542281EDF6
:101DF00096E00E94AE2560E471E080E090E00E94F1
:101E0000882810920E0161E081ED96E00E94542234
:101E100081ED96E00E94AE2560E471E080E090E004
:101E20000E94882864E170E080E090E00E948828A9
:101E30000E94FE0A8091CE069091CF060196909363
:101E4000CF068093CE0681ED96E00E94AE2580916C
:101E5000CE069091CF06889708F046C0CC24C39454
:101E6000D12C90E4E92EF12C00E410E020EB32E0DC
:101E700041E050E061E070E081ED96E00E94451F96
:101E800020E030E040E85EE36091000770910107D8
:101E900080910207909103070E94DF2D0E94F82C89
:101EA00001E010E09B0146E050E064E370E081ED6A
:101EB00096E00E94271E20E030E040E85EE360915B
:101EC00004077091050780910607909107070E940B
:101ED000DF2D0E94F82C9B0146E050E064E370E0A7
:101EE00081ED96E00E94271E8091CE069091CF064C
:101EF0008997C697D0F445E050E06AE070E081ED44
:101F000096E00E944E2268E081ED96E00E94542205
:101F10004AE050E06091D00681ED96E00E94D32A1D
:101F200061E081ED96E00E9454228091CE0690916E
:101F3000CF068036910508F4D4C04AE050E06AE04C
:101F400070E081ED96E00E944E2262E081ED96E025
:101F50000E94542280910A01803379F4E091C606F0
:101F6000F0E0EE0FFF1FE055F54F659174914AE0E8
:101F700050E081ED96E00E94DA2A80910A018133D7
:101F800079F4E091C506F0E0EE0FFF1FE055F54F44
:101F9000659174914AE050E081ED96E00E94DA2A62
:101FA00080910A01823379F4E091C406F0E0EE0FEB
:101FB000FF1FE055F54F659174914AE050E081EDC7
:101FC00096E00E94DA2A80910A01833379F4E09145
:101FD000C306F0E0EE0FFF1FE055F54F65917491D9
:101FE0004AE050E081ED96E00E94DA2A80910A01F1
:101FF000843379F4E091C206F0E0EE0FFF1FE05564
:10200000F54F659174914AE050E081ED96E00E94B1
:10201000DA2A80910A01853379F4E091C106F0E073
:10202000EE0FFF1FE055F54F659174914AE050E0C7
:1020300081ED96E00E94DA2A80910A01863379F4D4
:10204000E091C006F0E0EE0FFF1FE055F54F6591FF
:1020500074914AE050E081ED96E00E94DA2A809186
:102060000A01873379F4E091BF06F0E0EE0FFF1F1D
:10207000E055F54F659174914AE050E081ED96E0AE
:102080000E94DA2AE0910A01E03368F4F0E0EE0FF2
:10209000FF1FE055F54F659174914AE050E081EDE6
:1020A00096E00E94DA2A43E250E06AE070E081EDB7
:1020B00096E00E944E2264E875E081ED96E00E9471
:1020C000242A61E081ED96E00E9454228091CE06A0
:1020D0009091CF068437910520F01092CF06109290
:1020E000CE068090040790900507A0900607B09058
:1020F000070720E030E040EA51E4C501B4010E9446
:102100008C2C87FD12C0C0900007D0900107E09092
:102110000207F090030720E030E040EA51E4C701F5
:10212000B6010E948C2C87FF0BC04DE050E067E4A5
:1021300070E081ED96E00E944E2268E875E01EC0D6
:1021400020E030E04CE052E4C501B4010E94DB2DF8
:102150001816F4F420E030E04CE052E4C701B60178
:102160000E94DB2D1816A4F44DE050E067E470E007
:1021700081ED96E00E944E2262E975E081ED96E0E5
:102180000E94242A6AE070E080E090E00E948828A3
:1021900061E070E081ED96E00E945A2261E081EDFD
:1021A00096E00E94542240E050E062E070E081ED51
:1021B00096E00E944E226CE975E081ED96E00E9467
:1021C000242A4AE050E06091D00681ED96E00E941A
:1021D000D32A6EEA75E081ED96E00E94242A6AE037
:1021E00070E080E090E00E948828E091D106F091B4
:1021F000D2060684F785E02DEE24E394F12C02E06C
:1022000010E027E330E04BE150E068E470E081ED5E
:1022100096E00995C091D106D091D206609104074D
:102220007091050780910607909107070E94F82C8E
:10223000EE85FF859B014DE150E068E470E081EDA3
:1022400096E00995C091D106D091D2066091000721
:102250007091010780910207909103070E94F82C6A
:10226000EE85FF859B0142E250E068E470E081ED7D
:1022700096E00995E091D106F091D2060684F785A3
:10228000E02D27E330E044E250E068E470E081EDC7
:1022900096E00995E091D106F091D2062091CB0607
:1022A0003091CC060684F785E02DE12CF12C03E07B
:1022B00010E04DE150E068E470E081ED96E00995B2
:1022C000E091D106F091D2062091C9063091CA065C
:1022D0000684F785E02D42E250E068E470E081ED8D
:1022E00096E0099540E350E068E470E081ED96E007
:1022F0000E944E2280910A01803330F08F528093E9
:10230000D00661EB75E02AC0883230F087528093A6
:10231000D00667EB75E022C0803230F08F51809399
:10232000D0066DEB75E01AC0883130F0875180938C
:10233000D00664EC75E012C0803130F08F5080938D
:10234000D0066EEC75E00AC0883030F0875080937C
:10235000D00660ED75E002C062ED75E081ED96E0BB
:102360000E94242A81ED96E00E945E276AE070E0D8
:1023700080E090E00E94882880910A01883310F064
:1023800010920A0180910A01811103C087E38093B2
:102390000A01DF91CF911F910F91FF90EF90DF9095
:1023A000CF90BF90AF909F908F9008958AE00E9449
:1023B000BD2921E0892B09F420E020930D0188E05C
:1023C0000E94BD2921E0892B09F420E020930C0113
:1023D00083E00E94BD2921E0892B09F420E02093AD
:1023E0000B0180910D0181110BC080912001815062
:1023F0008093200164E670E080E090E00E948828ED
:1024000080910C01811108C010920E0164E670E009
:1024100080E090E00E94882880910B0181110BC020
:10242000809120018F5F8093200164E670E080E05E
:1024300090E00E948828809120018A3118F085E080
:102440008093200180912001853018F485E08093ED
:1024500020016091200182E090E00E94930881EDCC
:1024600096E00E94AE2561E081ED96E00E94542244
:1024700040E050E062E070E081ED96E00E944E2284
:1024800064ED75E081ED96E00E94242A44E150E07D
:102490006DE370E081ED96E00E944E224AE050E04C
:1024A0006091200181ED96E00E94D32A48E250E03D
:1024B00060E270E081ED96E00E944E228091200162
:1024C0008B3030F467EE75E081ED96E00E94242AAF
:1024D000809120018B50843030F462EF75E081ED03
:1024E00096E00E94242A809120018F3030F060E035
:1024F00076E081ED96E00E94242A81ED96E00E942C
:102500005E2760E08DE00C9487296091C60683E029
:1025100090E00E9493086091C50684E090E00E94DC
:1025200093086091C40685E090E00E949308609152
:10253000C30686E090E00E9493086091C20687E09F
:1025400090E00E9493086091C10688E090E00E94AC
:1025500093086091C00689E090E00E949308609122
:10256000BF068AE090E00C9493088AE00E94BD299F
:1025700021E0892B09F420E020930D0188E00E94DE
:10258000BD2921E0892B09F420E020930C0183E090
:102590000E94BD2921E0892B09F420E020930B0142
:1025A00080910D0181110BC08091BE0681508093F6
:1025B000BE0664E670E080E090E00E94882880918A
:1025C0000C01811144C084E080930E018091BE060D
:1025D000813029F480910A018093C60630C0823090
:1025E00029F480910A018093C50629C0833029F41B
:1025F00080910A018093C40622C0843029F480911E
:102600000A018093C3061BC0853029F480910A011A
:102610008093C20614C0863029F480910A01809309
:10262000C1060DC0873029F480910A018093C0064D
:1026300006C0883021F480910A018093BF0664E6C9
:1026400070E080E090E00E9488280E9485128091CE
:102650000B0181110BC08091BE068F5F8093BE0677
:1026600064E670E080E090E00E9488288091BE06D9
:10267000893018F081E08093BE068091BE068111FA
:1026800003C088E08093BE0681ED96E00E94AE25EF
:1026900061E081ED96E00E94542240E050E062E06B
:1026A00070E081ED96E00E944E226CE076E081EDD4
:1026B00096E00E94242A44E150E06DE370E081ED51
:1026C00096E00E944E224AE050E06091BE0681ED05
:1026D00096E00E94D32A81ED96E00E945E2760E09A
:1026E0008DE00C948729DF92EF92FF920F931F9356
:1026F000CF93DF9383E090E00E949108D82E8093DF
:10270000C60684E090E00E949108E82E8093C506FA
:1027100085E090E00E949108F82E8093C40686E040
:1027200090E00E949108082F8093C30687E090E014
:102730000E949108182F8093C20688E090E00E94C2
:102740009108D82F8093C10689E090E00E949108FB
:10275000C82F8093C0068AE090E00E949108809381
:10276000BF0697E39D1518F498E19093C60697E38A
:102770009E1518F49FE19093C50697E39F1518F4F2
:1027800098E19093C406083318F09FE19093C30634
:10279000183318F098E19093C206D83318F09FE1EF
:1027A0009093C106C83318F098E19093C00688331F
:1027B00018F08FE18093BF06DF91CF911F910F91A9
:1027C000FF90EF90DF900895CF92DF92EF92FF920B
:1027D0000F931F9361E08DE10E944E2961E08DE12E
:1027E0000E94872961E08DE00E944E2961E086E029
:1027F0000E944E2961E085E00E944E2961E080E15F
:102800000E944E2961E081E10E944E2961E08FE043
:102810000E944E2961E08DE00E94872921E04CE36F
:1028200062E081ED96E00E94292681ED96E00E940B
:10283000AE25CC24C394D12CF0E4EF2EF12C00E48F
:1028400010E020EB34E040E050E06EE170E081ED1C
:1028500096E00E94451F81ED96E00E945E2760EDA4
:1028600077E080E090E00E94882881ED96E00E9469
:10287000AE2561E070E081ED96E00E945A2261E0B1
:1028800081ED96E00E94542244E150E06AE070E05D
:1028900081ED96E00E944E2260E276E081ED96E0C6
:1028A0000E94242A48E250E06CE070E081ED96E05E
:1028B0000E944E2261E376E081ED96E00E94242A98
:1028C00081ED96E00E945E2761E081ED96E00E9436
:1028D00054226CED75E080E090E00E94882881ED44
:1028E00096E00E94AE2561E08DE00E94872964E1B8
:1028F00070E080E090E00E94882881E090E00E94F3
:10290000910880930A0182E090E00E9491088093F0
:1029100020016AE070E080E090E00E94882861E099
:1029200086E00E94872960E085E00E94872964E6AE
:1029300070E080E090E00E9488280E9402096AE02E
:1029400070E080E090E00E94882860E08AE00E94C9
:102950004E2962E08AE00E94872960E088E00E94B8
:102960004E2962E088E00E94872960E083E00E94AF
:102970004E2962E083E00E9487298AE00E94BD29F7
:1029800021E0892B09F420E020930D0188E00E94CA
:10299000BD2921E0892B09F420E020930C0183E07C
:1029A0000E94BD2921E0892B09F420E020930B012E
:1029B0001F910F91FF90EF90DF90CF900C947313C5
:1029C000BF92CF92DF92EF92FF920F931F93CF931C
:1029D000DF9381ED96E00E94AE251092C806D4E008
:1029E000BD2E8091C8068F3608F0F4C08F5F8093AB
:1029F000C806CC24C394D12CB0E4EB2EF12C00E417
:102A000010E020EB34E040E050E06EE170E081ED5A
:102A100096E00E94451F0E94FE0AE091D106F091C7
:102A2000D2060684F785E02DEE24E394F12C02E033
:102A300010E02CE730E04EE350E060E070E081ED24
:102A400096E00995E091D106F091D2060684F785CB
:102A5000E02D0FE310E021E030E040E050E061E0E5
:102A600070E081ED96E009950091D1061091D206B3
:102A70006091040770910507809106079091070700
:102A80000E94F82CD8011E96ED91FC911F970AE048
:102A900010E02AE030E0AB0162E070E081ED96E00A
:102AA0000995E091D106F091D2060684F785E02DD4
:102AB0000FE310E021E030E040E050E06CE070E037
:102AC00081ED96E00995E091D106F091D206068459
:102AD000F785E02D21E030E040E050E060E770E075
:102AE00081ED96E009950091D1061091D206609192
:102AF00000077091010780910207909103070E94DF
:102B0000F82CE801EE85FF850AE010E02AE030E0CD
:102B1000AB0161E770E081ED96E00995E091D106A7
:102B2000F091D2060684F785E02D0FE310E021E056
:102B300030E040E050E06BE770E081ED96E0099511
:102B4000D091C806DC30C8F10091D1061091D206B0
:102B5000609104077091050780910607909107071F
:102B60000E94F82CAD2FB0E0E801EE85FF8501E072
:102B700010E021E030E0AB01BD0181ED96E0099568
:102B80000091D1061091D206609100077091010763
:102B900080910207909103070E94F82CA091C8062B
:102BA000B0E0E801EE85FF8501E010E023E030E0D1
:102BB000AB01BD0181ED96E0099581ED96E00E94A3
:102BC0005E27B0920E0165E070E080E090E00E9428
:102BD000882807CFDF91CF911F910F91FF90EF9041
:102BE000DF90CF90BF900895DF92EF92FF920F9306
:102BF0001F93CF93DF9300D000D0CDB7DEB7DD2495
:102C0000D3948091FF0681110BC28AE00E94BD29F6
:102C100021E0892B09F420E020930D0188E00E9437
:102C2000BD2921E0892B09F420E020930C0183E0E9
:102C30000E94BD2921E0892B09F420E020930B019B
:102C40000E94FE0A80910D0181111EC080910B012E
:102C500081111AC081ED96E00E94AE2540E250E05D
:102C600062E270E081ED96E00E944E2261E476E03F
:102C700081ED96E00E94242A81ED96E00E945E2775
:102C800084E080930E01CCC120E030E048E452E4BF
:102C900060910407709105078091060790910707DE
:102CA0000E94DB2D181684F020E030E048E452E466
:102CB00060910007709101078091020790910307CE
:102CC0000E94DB2D181614F4D092FF0664E170E028
:102CD00080E090E00E94882845E350E06DE270E0DB
:102CE00081ED96E00E944E22409104075091050725
:102CF000609106077091070722E030E081ED96E0D1
:102D00000E94CB2B60910407709105078091060704
:102D1000909107070E94F82C9B01AC0181ED96E091
:102D200029833A834B835C830E94672229813A81FD
:102D300097FD01969595879501E010E0AC0169E15A
:102D400070E081ED96E00E94271E20E030E040E038
:102D50005FE36091040770910507809106079091E9
:102D600007070E94DF2D0E94F82C9B01AC0181ED2A
:102D700096E029833A834B835C830E9467222981F2
:102D80003A8197FD01969595879501E010E0AC0199
:102D900069E170E081ED96E00E94271E20E030E0BE
:102DA00040EA50E46091040770910507809106079E
:102DB000909107070E94902C0E94F82C9B01AC0177
:102DC00081ED96E029833A834B835C830E946722DE
:102DD00029813A8197FD01969595879501E010E04C
:102DE000AC0169E170E081ED96E00E94271E81ED63
:102DF00096E00E945E276FE070E080E090E00E9425
:102E0000882881ED96E00E94AE2545E350E06DE212
:102E100070E081ED96E00E944E22409104075091AF
:102E20000507609106077091070722E030E081ED09
:102E300096E00E94CB2B6091000770910107809172
:102E40000207909103070E94F82C9B01AC0181EDD1
:102E500096E029833A834B835C830E946722298111
:102E60003A8197FD01969595879501E010E0AC01B8
:102E700066E670E081ED96E00E94271E20E030E0DB
:102E800040E05FE3609100077091010780910207C5
:102E9000909103070E94DF2D0E94F82C9B01AC014A
:102EA00081ED96E029833A834B835C830E946722FD
:102EB00029813A8197FD01969595879501E010E06B
:102EC000AC0166E670E081ED96E00E94271E20E0EE
:102ED00030E040EA50E46091000770910107809172
:102EE0000207909103070E94902C0E94F82C9B01EE
:102EF000AC0181ED96E029833A834B835C830E9489
:102F0000672229813A8197FD01969595879501E081
:102F100010E0AC0166E670E081ED96E00E94271EAD
:102F200081ED96E00E945E276FE070E080E090E027
:102F30000E94882881ED96E00E94AE2545E350E08E
:102F40006DE270E081ED96E00E944E224091040710
:102F500050910507609106077091070722E030E065
:102F600081ED96E00E94CB2B0091D1061091D20604
:102F7000209100073091010740910207509103070B
:102F800060910407709105078091060790910707EB
:102F90000E94272C0E94F82CD8011E96ED91FC91DE
:102FA0001F97EE24E394F12C06E010E025E030E0DA
:102FB000AB0167E170E081ED96E009950091D106E3
:102FC0001091D20620910407309105074091060721
:102FD00050910707609100077091010780910207E7
:102FE000909103070E94272C0E94F82CD8011E966E
:102FF000ED91FC911F9706E010E025E030E0AB0179
:1030000064E670E081ED96E0099581ED96E00E941E
:103010005E276FE070E080E090E00E948828F1CDAC
:103020001092FF060F900F900F900F90DF91CF91AD
:103030001F910F91FF90EF90DF900895CF92DF9254
:10304000EF92FF920F931F930E94990981ED96E0F2
:103050000E94AE25CC24C394D12CA0E4EA2EF12CFE
:1030600000E410E020EB30E040E050E06EE170E082
:1030700081ED96E00E94451F1F910F91FF90EF9008
:10308000DF90CF900895CF92DF92EF92FF920F934F
:103090001F938091BA069091BB068536910590F1F9
:1030A0000E941E1889E690E09093BB068093BA06B2
:1030B0008AE00E94BD2921E0892B09F420E02093B9
:1030C0000D0188E00E94BD2921E0892B09F420E050
:1030D00020930C0183E00E94BD2921E0892B09F493
:1030E00020E020930B0180910D01882331F0809125
:1030F0000C01882311F0211164C11092BB061092BB
:10310000BA065FC10E9499098091BA069091BB06E8
:1031100001969093BB068093BA0680910E01813090
:1031200041F41F910F91FF90EF90DF90CF900C949E
:10313000F415823041F41F910F91FF90EF90DF90D2
:10314000CF900C94D611833041F41F910F91FF90D2
:10315000EF90DF90CF900C94E014843041F41F91F5
:103160000F91FF90EF90DF90CF900C94310C853051
:1031700041F41F910F91FF90EF90DF90CF900C944E
:10318000B5128AE00E94BD2921E0892B09F420E0D4
:1031900020930D0188E00E94BD2921E0892B09F4CC
:1031A00020E020930C0183E00E94BD2921E0892BBF
:1031B00009F420E020930B0180910D01811109C0D9
:1031C00080910F01815080930F011092BB061092E5
:1031D000BA0690910C0180910F01911106C0809365
:1031E0000E011092BB061092BA06211107C08F5F24
:1031F00080930F011092BB061092BA0680910F01C6
:10320000853018F081E080930F0180910F018111CA
:1032100003C081E080930F0181ED96E00E94AE250E
:10322000CC24C394D12C10E4E12EF12C00E810E062
:1032300020EB36E040E050E060E070E081ED96E0A9
:103240000E94451F61E081ED96E00E94542240916A
:103250000F01E091D106F091D2068AE0489FA001CB
:1032600011244D5F5F4F0684F785E02DEE24E39433
:10327000F12C0AE010E028E730E063E070E081ED37
:1032800096E0099561E070E080910F01811102C024
:1032900060E070E081ED96E00E945A2241E050E04B
:1032A00060E070E081ED96E00E944E2287EA90E0B7
:1032B0000E949508BC0181ED96E00E94242A61E0FD
:1032C00070E080910F01813011F460E070E081EDD9
:1032D00096E00E945A224FE050E062E070E081EDFB
:1032E00096E00E944E2288E990E00E949508BC0179
:1032F00081ED96E00E94242A61E070E080910F0148
:10330000823011F460E070E081ED96E00E945A2274
:1033100049E150E062E070E081ED96E00E944E22CB
:1033200085E890E00E949508BC0181ED96E00E943E
:10333000242A61E070E080910F01833011F460E095
:1033400070E081ED96E00E945A2243E250E062E094
:1033500070E081ED96E00E944E2287E790E00E94A7
:103360009508BC0181ED96E00E94242A61E070E09E
:1033700080910F01843011F460E070E081ED96E0FF
:103380000E945A224DE250E062E070E081ED96E04A
:103390000E944E2288E690E00E949508BC0181EDD3
:1033A00096E00E94242A81ED96E00E945E2760E06C
:1033B0008DE01F910F91FF90EF90DF90CF900C94D4
:1033C00087291F910F91FF90EF90DF90CF90089584
:1033D00064E081ED96E00C9495258091380790E0AB
:1033E00020913907821B9109089520913907809116
:1033F0003807281750F4E22FF0E0E65CF84F8081A0
:1034000090E02F5F2093390708958FEF9FEF089585
:10341000E091390780913807E81730F4F0E0E65C76
:10342000F84F808190E008958FEF9FEF0895089501
:10343000CF92DF92EF92FF920F931F93CF93DF9380
:103440007C01CB018A0120911407222389F0EB0132
:103450006B01C40ED51ECC15DD0569F06991D7014D
:10346000ED91FC910190F081E02DC7010995F3CF1A
:10347000642F0E94291BC801DF91CF911F910F91EA
:10348000FF90EF90DF90CF900895CF93DF931F923E
:10349000CDB7DEB76983209114072223D1F02091A4
:1034A0001507203240F021E030E0FC013383228315
:1034B00080E090E015C080911607E82FF0E0E95E0B
:1034C000F84F998190838F5F80931607809315073B
:1034D00005C061E0CE0101960E94291B81E090E0C9
:1034E0000F90DF91CF910895FC011382128248EE74
:1034F00053E060E070E044835583668377838FE414
:1035000096E09183808308951092390710923807CE
:1035100010921607109215070C94B41A81E080934C
:103520001407609337071092160710921507089535
:103530000C948E1A0F93062F21E04091150767E136
:1035400077E0809137070E94D21A109216071092E6
:103550001507109214070F91089561E00C949A1AC0
:1035600088E097E00C94741A1092C70781E080936A
:10357000C5071092C40761E082E10E94872961E0DB
:1035800083E10E948729E9EBF0E080818E7F8083D0
:1035900080818D7F808388E48093B80085E4809368
:1035A000BC0008950F93413208F04AC09091C707BC
:1035B0009111FCCF92E09093C7070093C5079FEF4E
:1035C00090935A0710929F0740939E07FB0160EA71
:1035D00077E0DB019A2F961B941718F491919D9335
:1035E000F9CF1092C6079091C607880F892B809358
:1035F000C6078091C407813061F41092C40780919E
:10360000C6078093BB008091BC0083FDF8CF85EC9A
:1036100001C085EE8093BC00222321F08091C70772
:103620008230E1F380915A078F3F61F080915A0711
:10363000803251F080915A07803341F483E007C013
:1036400081E005C080E003C082E001C084E00F910A
:103650000895613298F42091C707243089F460936B
:103660007C07FC018EE797E0DC012A2F281B261738
:1036700018F421912D93F9CF80E0089581E0089509
:1036800082E0089585ED8093BC008091BC0084FDAC
:10369000FCCF1092C707089585EC8093BC00109270
:1036A000C70708951F920F920FB60F9211242F9300
:1036B0003F934F935F936F937F938F939F93AF93BA
:1036C000BF93EF93FF938091B900887F803609F410
:1036D0009EC078F5883209F45DC090F4803109F419
:1036E00056C038F4882309F4F5C0883009F44FC077
:1036F000F5C0883109F44EC0803209F45FC0EEC0D5
:10370000803409F46AC058F4803309F457C0883310
:1037100009F0E4C080935A070E944C1BDFC080353B
:1037200009F44FC0883509F45DC0883409F0D6C06B
:10373000D3C0883909F4C4C0A8F4883709F467C035
:1037400038F4883609F463C0803709F460C0C6C015
:10375000883809F4B5C0803909F45FC0803809F0B1
:10376000BDC05BC0803B09F483C038F4803A09F4E3
:1037700066C0883A09F47CC0B1C0803C09F4A4C09A
:10378000883C09F4A1C0883B09F487C0A7C0809198
:10379000C60710C090919F0780919E07981770F5FB
:1037A000E0919F0781E08E0F80939F07F0E0E05645
:1037B000F84F80818093BB0085EC83C080935A07CB
:1037C0008BC0E0919F0781E08E0F80939F078091CF
:1037D000BB00F0E0E056F84F808390919F07809106
:1037E0009E076BC0E0919F0781E08E0F80939F073B
:1037F0008091BB00F0E0E056F84F80838091C507D0
:1038000081116AC081E08093C40784EA5EC083E0CE
:103810008093C70710925B07CFCF80915B07803200
:1038200008F04EC0E0915B0781E08E0F80935B074C
:103830008091BB00F0E0E45AF84F8083BDCF0E9436
:103840004C1B80915B07803230F4E0915B07F0E025
:10385000E45AF84F108260915B0770E0E091C00776
:10386000F091C1078CE597E0099510925B0736C08F
:1038700084E08093C70710927D0710927C07E09147
:10388000C207F091C307099580917C07811105C09B
:1038900081E080937C0710927E07E0917D0781E0B4
:1038A0008E0F80937D07F0E0E258F84F808180937F
:1038B000BB0090917D0780917C07981708F47CCF1E
:1038C00085E88093BC000AC085EC8093BC00109210
:1038D000C70704C010925A070E94421BFF91EF9144
:1038E000BF91AF919F918F917F916F915F914F9118
:1038F0003F912F910F900FBE0F901F9018952F9210
:103900003F924F925F926F927F928F929F92AF926F
:10391000BF92CF92DF92EF92FF920F931F93CF93BC
:10392000DF9300D000D0CDB7DEB74C017C836B8332
:103930006A015901C8018701AC014C195D0957FFA3
:1039400003C051954195510995016B817C81261BDE
:10395000370B37FF03C03195219531092224239479
:10396000312C2417350714F0212C312C211431046B
:1039700059F03A2D2B2D5C01832F922F3B812C8106
:10398000DC82CB82C32ED22EAB81BC81AA16BB06B1
:103990005CF43C2D2D2D6C01832F922F3B812C81CB
:1039A000BC82AB82A32EB22E2501EB81FC814E1A84
:1039B0005F0A3C016C187D0877FE03C07194619426
:1039C0007108720157FE03C0FFEFEF1AFF0AF5946A
:1039D000E794C816D9062CF421E030E03A83298315
:1039E00024C06FEF7FEF7A8369831FC0D401ED910C
:1039F000FC910480F581E02D980121143104D9F067
:103A00004B815C81B601C4010995E618F708F7FE01
:103A100006C0E981FA81CE0EDF1EE40CF51C2B8175
:103A20003C812F5F3F4F3C832B836B817C81A616AB
:103A3000B706E4F604C0A6016B817C81E4CF0F9049
:103A40000F900F900F90DF91CF911F910F91FF90EA
:103A5000EF90DF90CF90BF90AF909F908F907F902E
:103A60006F905F904F903F902F9008956F927F924C
:103A70008F929F92AF92BF92CF92DF92EF92FF927E
:103A80000F931F93CF93DF93EC015B016A01390120
:103A90004801E881F9810284F385E02D87010995C9
:103AA000E881F981A601480D591D41505109028450
:103AB000F385E02D9301B501CE010995E881F981E7
:103AC0000084F185E02D9401A601B501CE01099590
:103AD000E881F981B501660D771D61507109008497
:103AE000F185E02D9401A601CE010995DF91CF91DA
:103AF0001F910F91FF90EF90DF90CF90BF90AF900C
:103B00009F908F907F906F900895EF92FF920F9308
:103B10001F93DC01ED91FC91240F351F21503109D9
:103B20000680F781E02D780189019B0109951F919D
:103B30000F91FF90EF900895EF92FF920F931F93D4
:103B4000DC01ED91FC91260F371F215031090680D1
:103B5000F781E02D78018A0109951F910F91FF905F
:103B6000EF9008956F927F928F929F92AF92BF9243
:103B7000CF92DF92EF92FF920F931F93CF93DF9339
:103B80005C014A0169013801EB01C60ED71ECC1554
:103B9000DD0574F4D501ED91FC910084F185E02DF3
:103BA00087019301A401BE01C50109952196EFCFBC
:103BB000DF91CF911F910F91FF90EF90DF90CF9009
:103BC000BF90AF909F908F907F906F900895EF92ED
:103BD000FF920F931F93DC01ED91FC9111971A96C0
:103BE0000D911C911B9718962D913C911997068465
:103BF000F785E02D7B0140E050E060E070E0099542
:103C00001F910F91FF90EF9008950895FC0113828A
:103C100012828FE596E09183808375836483578356
:103C200046837187608753874287158A1586148675
:103C30001786168621E0248B8FEF9FEF938B828B64
:103C4000918B808B268B178A118E108E08952F9260
:103C50003F924F925F926F927F928F929F92AF921C
:103C6000BF92CF92DF92EF92FF920F931F93CF9369
:103C7000DF9300D000D000D0CDB7DEB79E838D8318
:103C80006B015A01790166246394712C621A730ADC
:103C900044245524421A530A440C551CDC01ED916E
:103CA000FC91420F531F0480F581E02D9801099586
:103CB000AD81BE81ED91FC911197A5014E195F096F
:103CC0000480F581E02D9801B601CD010995AD8103
:103CD000BE81ED91FC911197B6016E0D7F1D0480A0
:103CE000F581E02D9801A501CD010995AD81BE8139
:103CF000ED91FC911197B6016E197F090480F58151
:103D0000E02D9801A501CD010995812C912C8E14EF
:103D10009F040CF0A1C077FC08C0B1E0EB1AF108D9
:103D2000E2E04E0E511C640C751CFFEF8F1A9F0AC7
:103D3000C401880F991F0196680E791EC4018C0D6D
:103D40009D1D9C838B83AD81BE81ED91FC9111976C
:103D50000480F581E02D980115012E0C3F1CA10176
:103D6000BC01CD010995F601E819F909FA83E98347
:103D7000AD81BE81ED91FC9111970480F581E02D1C
:103D80009801A10169817A81CD010995AD81BE813A
:103D9000ED91FC9111970480F581E02D98011501BA
:103DA0002E183F08A1016B817C81CD010995AD8161
:103DB000BE81ED91FC9111970480F581E02D980171
:103DC000A10169817A81CD01099514012A0C3B1C5E
:103DD000AD81BE81ED91FC9111970480F581E02DBC
:103DE0009801A101C6018E0D9F1D9C838B83BC0190
:103DF000CD010995AD81BE81ED91FC9111970480B3
:103E0000F581E02D9801A101C6018E199F099A83C1
:103E10008983BC01CD010995150128183908AD81A8
:103E2000BE81ED91FC9111970480F581E02D980100
:103E3000A1016B817C81CD010995AD81BE81ED91A0
:103E4000FC9111970480F581E02D9801A101698111
:103E50007A81CD0109955BCF26960FB6F894DEBF27
:103E60000FBECDBFDF91CF911F910F91FF90EF90CB
:103E7000DF90CF90BF90AF909F908F907F906F908A
:103E80005F904F903F902F9008952F923F924F92C6
:103E90005F926F927F929F92AF92BF92CF92DF928A
:103EA000EF92FF920F931F93CF93DF93CDB7DEB7BF
:103EB0002A970FB6F894DEBF0FBECDBF5C017C839E
:103EC0006B835E834D83190127013601C801079674
:103ED00097FD07969C0193E0359527959A95E1F714
:103EE0003A832983C12CD12CE12CF12CE414F50464
:103EF0000CF044C01A8619868D819E818E0D9F1DFF
:103F000098878F83E985FA85E017F1077CF5898525
:103F10009A8587709927892B11F0990C0EC0E98535
:103F2000FA85F7FD379683E0F595E7958A95E1F7F1
:103F3000EC0DFD1DE20DF31D949097FE11C0D5010F
:103F4000ED91FC910480F581E02D93014F8158851E
:103F50006B817C8189859A85680F791FC5010995D8
:103F6000A985BA851196BA87A987CCCFFFEFEF1A3A
:103F7000FF0A29813A81C20ED31EB8CF2A960FB606
:103F8000F894DEBF0FBECDBFDF91CF911F910F918F
:103F9000FF90EF90DF90CF90BF90AF909F907F9079
:103FA0006F905F904F903F902F9008952F923F9287
:103FB0004F925F926F927F928F929F92AF92BF9239
:103FC000CF92DF92EF92FF920F931F93CF93DF93E5
:103FD000CDB7DEB76A970FB6F894DEBF0FBECDBF80
:103FE0001C0158874F831C870B87FA86E986CC8291
:103FF000DC0158964D915C9159974115510509F096
:10400000A6C018968D919C911997681779070CF0A6
:1040100056C11A968D919C911B97EF81F885E817F0
:10402000F9070CF04CC1D12CCB013C81F6E03F9F4D
:10403000800D911D1124181619060CF040C1C601FF
:1040400003E0880F991F0A95E1F74F815885840F87
:10405000951F181619060CF032C157968C918111D4
:1040600003C0203B08F02F5F7E876D874B011982CC
:1040700010E7A12E1BE0B12EA61AB70A55E0259F26
:10408000A00CB11C11248981853039F0ED85FE85A5
:10409000EA0DFB1D94919A8301C01A826F80788487
:1040A0002301A8E0AD83BA81B0FF12C0D101ED9128
:1040B000FC91BC81B13031F40480F581E02D2B8579
:1040C0003C8518C00684F785E02DEB84FC841DC078
:1040D000E985FA852B853C85E217F307E1F0D101EC
:1040E000ED91FC91BC81B13059F40480F581E02D53
:1040F00029853A85A2016D857E85C10109950BC090
:104100000684F785E02DE984FA8486019601A301EF
:10411000B401C1010995EA81E695EA83FD81F15078
:10412000FD836C0C7D1C2FEF421A520AF111BBCF9C
:1041300039813F5F39838C0C9D1C4D855E854F5FB7
:104140005F4F5E874D87363009F09DCFB8C0FA01CA
:1041500034963491329785919491231BA7E02A9F3E
:10416000800D911D1124FA0125913491398B288BF2
:10417000FC01459154915A8F498FFC01329654911C
:1041800059873196A491AF873196E491FC01359619
:10419000249131968491BC81B23050F0622E772404
:1041A00067FC7094E82FFF27E7FDF095FE87ED8709
:1041B000FC81CF2ED12C6C9C40016D9C900C7C9C82
:1041C000900C1124860E971EA12C1982DE8ACD8AAE
:1041D000AB01420F511D27FD5A955E834D83AF8180
:1041E000B885A80FB11D87FDBA95B88FAF8B5981DF
:1041F0008F85581708F063C0852F90E02D853E8588
:10420000280F391F2C9DD0012D9DB00D3C9DB00D68
:104210001124EF81F885EA0FFB1FFB83EA836D8091
:104220007E802401FA2D2D81F21BFA8B4F89588D47
:10423000480F591F5C8B4B8B9A89960D862D2D81CB
:10424000821B39858317B0F5977061F4898D9A8D3B
:104250000196E889F989298D3A8DE20FF31FB49010
:104260009A8F898FB7FE1DC0D101ED91FC91BC8161
:10427000B13059F40480F581E02D2B853C854B89C4
:104280005C89B301C10109950CC00684F785E02D56
:10429000EB84FC84860196014A815B81B201C101F5
:1042A0000995BB0CED89FE894E0E5F1EFFEF6F1A5C
:1042B0007F0AC2CFA30E49814F5F498398CF6A9688
:1042C0000FB6F894DEBF0FBECDBFDF91CF911F9127
:1042D0000F91FF90EF90DF90CF90BF90AF909F90A5
:1042E0008F907F906F905F904F903F902F900895A8
:1042F000AF92BF92CF92EF92FF920F931F93CF9303
:10430000DF93EC01262F888D998D009709F042C02C
:104310006A3069F42C898E859F8538E0239F800D53
:10432000911D11249F878E871D861C86ABC06D3022
:1043300009F4A8C08E898823C1F03C898C859D85AD
:1043400046E0349F800D911D1124488559858417BE
:1043500095075CF01D861C868E859F85E8E03E9F54
:10436000800D911D11249F878E87EA88FB8808891C
:1043700019894E855F856C857D85CC88CE010E942C
:10438000D61F2C898C859D85F6E02F9F800D911D71
:10439000112441C06A3079F41D861C864C89FC01C9
:1043A000369684912E853F85489F200D311D11241E
:1043B0003F872E8767C06D3009F464C0AC014C5F45
:1043C0005F4FFA013491631708F45CC03196E491B1
:1043D000E61708F457C0FA014491362F341BFC014C
:1043E0003296A590B490F7E03F9FA00CB11C112429
:1043F000F5013296A4913196E491AA2311F0E111CE
:104400000DC0F5013496A4902C898C859D85A29EC3
:10441000800D911D11249D878C8734C0F501359640
:10442000E4913E89332309F13C89B0E0AE0FB11D20
:10443000E7FDBA953A9FA0013B9F500D11246C8572
:104440007D85460F571F68857985461757076CF09D
:104450001D861C86FC01369684914E855F85389FAB
:10446000400D511D11245F874E87EA88FB8808891B
:1044700019894E855F856C857D85CC88CE010E942B
:10448000D61FBFCF81E090E0DF91CF911F910F91B8
:10449000FF90EF90CF90BF90AF900895FC0175878B
:1044A0006487578746870895611101C061E0FC0168
:1044B000648B0895FC01738B628B718B608B089504
:1044C000FC0185890895FC01808591850895FC0192
:1044D0008285938508950F931F93CF93DF93EC010B
:1044E0008D89823061F08330D9F0813009F0C8C005
:1044F000EC81FD81E41BF50B3197DB0118C08C8149
:104500009D81DC01A61BB70BBD018E819F81FC0143
:10451000E41BF50BAF0141505109621B730BB0C096
:10452000AE81BF81A61BB70BA21BB30BFA01F7FD2F
:1045300005C18C819D81E817F9070CF0FFC0B7FF1A
:1045400004C02A0F3B1FA0E0B0E08E819F81AD0127
:10455000420F531F841795071CF49C012A1B3B0B29
:10456000121613060CF0EAC0422F8A2F8695869504
:10457000869590E8899FE00DF11D1124EE5CFE4FB9
:10458000A77069F158E05A1B852F90E0EC01C65DD9
:10459000DE4F6881251760F4DC01A21BB1098FEFA3
:1045A00090E00A2E02C0959587950A94E2F7682359
:1045B0000130110539F048F00230110551F48081C5
:1045C000862706C08081862B03C060958081862364
:1045D0008083451708F4B2C0451BE058FF4F4830B0
:1045E000A0F102301105A9F4DF01842F9C91909570
:1045F0009C93A058BF4F88508830C0F788EF840F35
:10460000869586958695B0E88B9FE00DF11D112467
:1046100019C081E00130110509F080E0982F9195D3
:10462000EF01842F9883C058DF4F88508830D0F72F
:1046300088EF840F86958695869590E8899FE00D92
:10464000F11D1124E058FF4F4770442309F476C050
:10465000A42FB0E0AE5DBE4F9C910130110541F03A
:1046600050F00230110509F069C08081892706C029
:104670008081892B03C090958081892380835EC0CF
:1046800057FD5CC08E819F81481759070CF056C0BA
:1046900077FF04C0260F371F60E070E08C819D819A
:1046A000FB01E20FF31F8E179F071CF49C01261BD2
:1046B000370B121613060CF041C0CA0157FD0796BE
:1046C000E3E095958795EA95E1F79695982F8827E9
:1046D000979587958E5C9E4F860F971F477055273D
:1046E00061E070E001C0660F4A95EAF7462F01309D
:1046F000110541F088F00230110501F5FC01280F89
:10470000391F15C0FC01280F391FE217F307B1F05C
:104710008081842B8193F9CF6095FC01280F391F8C
:10472000E217F30759F0808186238193F9CFE217CE
:10473000F30721F0808184278193F9CFDF91CF9116
:104740001F910F9108950F931F93CF93DF93FC0157
:104750008589823069F08330E1F0813009F082C0D0
:10476000C481D581C41BD50BC21BD30BDB0117C081
:1047700084819581DC01A61BB70BBD0161507109D5
:1047800086819781DC01A41BB50BAD01421B530B45
:1047900069C0A681B781A61BB70B1197EA01B7FDC7
:1047A00008C186819781A817B9070CF002C1D7FF0D
:1047B00004C02C0F3D1FC0E0D0E084819581AE0184
:1047C000420F531F841795071CF49C012C1B3D0BB3
:1047D000121613060CF0EDC0CD01B7FD079643E0AD
:1047E000959587954A95E1F79695982F88279795FF
:1047F00087958E5C9E4F8C0F9D1FA770BB2741E055
:1048000050E00A2E01C0440F0A94EAF7642F0130E9
:10481000110549F098F00230110509F0CAC0FC01F9
:10482000280F391F17C0FC01280F391FE217F307A3
:1048300009F4BFC08081862B8193F8CF4095FC019D
:10484000280F391FE217F30709F4B3C080818423CE
:104850008193F8CFE217F30709F4ABC08081862774
:104860008193F8CF77FDA5C084819581681779077A
:104870000CF09FC057FF04C0240F351F40E050E0EC
:1048800086819781FA01E20FF31F8E179F071CF4B0
:104890009C01241B350B121613060CF08AC0522FF4
:1048A000842F869586958695FB01B0E88B9FE00D59
:1048B000F11D1124EE5CFE4F477069F168E0641B46
:1048C000862F90E0EC01C65DDE4F4881261760F42C
:1048D000DC01A21BB1098FEF90E00A2E02C0959572
:1048E00087950A94E2F748230130110539F048F022
:1048F0000230110551F48081842706C08081842B09
:1049000003C04095808184238083561708F451C0EA
:10491000561BE058FF4F5830A0F102301105A9F4A2
:10492000DF01852F9C9190959C93A058BF4F885094
:104930008830C0F788EF850F869586958695B0E814
:104940008B9FE00DF11D112419C081E0013011058C
:1049500009F080E0982F9195EF01852F9883C0583A
:10496000DF4F88508830D0F788EF850F8695869581
:10497000869590E8899FE00DF11D1124E058FF4FC6
:1049800057705523B1F0A52FB0E0AE5DBE4F9C919E
:104990000130110539F048F00230110551F48081E1
:1049A000892706C08081892B03C090958081892347
:1049B0008083DF91CF911F910F910895CF92DF9265
:1049C000EF92FF920F931F93CF93DF937C018B01A4
:1049D000EA01690177FDA0C00E9463220817190748
:1049E0000CF09AC0D7FD98C0C7010E946722C81773
:1049F000D9070CF091C0C7010E946022823009F0F3
:104A00007FC0F701848195819C01201B310B8901B6
:104A10000150110986819781FC01EC1BFD0BEF0110
:104A200021970BC0813049F4F701848195818C1B5B
:104A30009D0BE8018C0101501109F1E0CF16D10462
:104A400031F010F132E0C316D104E1F165C0FE018E
:104A5000D7FD379683E0F595E7958A95E1F7F695CA
:104A6000FE2FEE27F795E795E00FF11FEE5CFE4F66
:104A7000C770DD2781E090E00C2E01C0880F0A94FA
:104A8000EAF79081982B3AC0FE01D7FD3796A3E054
:104A9000F595E795AA95E1F7F695FE2FEE27F795A0
:104AA000E795E00FF11FEE5CFE4FC770DD2781E058
:104AB00090E00C2E01C0880F0A94EAF7809590814F
:104AC00098231CC0FE01D7FD379663E0F595E79566
:104AD0006A95E1F7F695FE2FEE27F795E795E00F3B
:104AE000F11FEE5CFE4FC770DD2781E090E00C2ED9
:104AF00001C0880F0A94EAF79081982790830CC030
:104B0000833009F08FCFF70186819781801B910B4D
:104B10008E01EC01219791CFDF91CF911F910F91E1
:104B2000FF90EF90DF90CF9008951F93CF93DF9386
:104B3000EC01162F40E450E060E870E00E94061E91
:104B400087E796E0998388838FEF8C8F88A38E8F79
:104B50008D8F1F8FDF91CF911F91089580E094E09A
:104B6000E2E3F1E0DF019C011D9221503040E1F7CA
:104B70000895FC0181A1882339F06EBD00000DB4B9
:104B800007FEFDCF8EB5089588E090E030E8A4A13F
:104B9000B5A14C9123A5209524232C93A2A1B3A1C8
:104BA00022A5432F462321F04C91422B4C9304C065
:104BB0004C91209524232C93A4A1B5A12C9143A51D
:104BC000242B2C933695019711F708951F93CF93BB
:104BD000DF93EC01162F8C8D8F3F09F1EEA1FFA121
:104BE00080819CA5892B8083E8A5F9A590818DA55E
:104BF000809589238083EEA1FFA190818CA580956B
:104C000089238083CE010E94B925EEA1FFA1808176
:104C10009CA5892B8083DF91CF911F9108958A8D68
:104C2000682F772767FD709588E097E00E94981AB3
:104C300060E088E097E00E94451A612F88E097E0E5
:104C40000E94451A88E097E0DF91CF911F910C9464
:104C5000AD1A0F931F93CF93DF93EC01162F022F02
:104C60006B8F4A8F8C8D8F3F09F48CC061E08E8DE5
:104C70000E944E2961E088A10E944E2988A19927AF
:104C800087FD9095FC01E856FF4EE491F0E0EE0FB1
:104C9000FF1FEA54FF4E259134913FA32EA3FC0140
:104CA000EC57FF4E84918CA78E8D992787FD9095A8
:104CB000FC01E856FF4EE491F0E0EE0FFF1FEA54CE
:104CC000FF4E2591349139A728A7FC01EC57FF4EE0
:104CD00084918DA789A1811134C061E08C8D0E94DF
:104CE0004E2961E08D8D0E944E298D8D992787FD7B
:104CF0009095FC01E856FF4EE491F0E0EE0FFF1FA7
:104D0000EA54FF4E259134913DA32CA3FC01EC57AE
:104D1000FF4E84918BA78C8D992787FD9095FC0180
:104D2000E856FF4EE491F0E0EE0FFF1FEA54FF4E0D
:104D3000259134913BA32AA3FC01EC57FF4E8491AB
:104D40008AA789A1882311F10E94E5278091CA07CB
:104D5000882399F09FB7F8948091CA07813059F45D
:104D60008DB38093C8072DB38091C90780958223A6
:104D70008DBB9FBF02C09093C80780E58CBD81E0CA
:104D80008DBD04C088E097E00E94841A0023F1F0F2
:104D90008F8D87FD1BC061E00E944E2961E08F8DE1
:104DA0000E94872961E070E080E090E00E948828FE
:104DB00060E08F8D0E9487296AE070E080E090E0DB
:104DC0000E94882861E08F8D0E9487296EEACE01BB
:104DD0000E94E62565EDCE010E94E62560E8CE0141
:104DE0000E94E62568EACE010E94E6256FE3CE0127
:104DF0000E94E62563EDCE010E94E62560E0CE012B
:104E00000E94E62560E4CE010E94E6256DE8CE0111
:104E10000E94E625113011F460E101C064E1CE0189
:104E20000E94E62560E2CE010E94E62560E0CE0108
:104E30000E94E62561EACE010E94E62568ECCE01DB
:104E40000E94E6256AEDCE010E94E62562E1CE01D0
:104E50000E94E62561E8CE010E94E625113011F49A
:104E60006FE901C06FECCE010E94E62569EDCE012D
:104E70000E94E625113011F462E201C061EFCE011B
:104E80000E94E6256BEDCE010E94E62560E4CE018E
:104E90000E94E62564EACE010E94E62566EACE017C
:104EA0000E94E6256EE2CE010E94E6256FEACE0161
:104EB000DF91CF911F910F910C94E625DF92EF9235
:104EC000FF920F931F93CF93DF93EC0161E20E9457
:104ED000E62560E0CE010E94E6256FE7CE010E9444
:104EE000E62562E2CE010E94E62560E0CE010E9446
:104EF000E62567E0CE010E94E6258C8D8F3F31F1DB
:104F0000EEA1FFA180819CA5892B8083E8A5F9A54E
:104F100080819DA5892B8083EEA1FFA190818CA526
:104F200080958923808302E311E0F80161918F016C
:104F3000CE010E94B925F5E002331F07B1F7EEA1BB
:104F4000FFA180819CA5892B808337C0D090B800B9
:104F50008CE08093B80002E311E06A8D772767FD4B
:104F6000709588E097E00E94981AE0910807F09108
:104F700009070190F081E02D60E488E097E0099551
:104F8000E12CF12CF801EE0DFF1D608188E097E027
:104F90000E94451A8FEFE81AF80AE0E1EE16F104D4
:104FA00089F788E097E00E94AD1A005F1F4FF5E097
:104FB00002331F0791F6D092B800DF91CF911F9175
:104FC0000F91FF90EF90DF900895CF93CFB7F894B3
:104FD0008091CB07811127C0E2EAF0E18491EEE8ED
:104FE000F0E19491E82FF0E0EE0FFF1FE054FF4E48
:104FF000A591B4918C91892321F461E08AE00E940B
:10500000872961E08AE00E944E298CB580618CBDC1
:105010008CB580648CBD61E08DE00E944E2961E01A
:105020008BE00E944E298091CB078F5F8093CB0746
:10503000CFBFCF9108951F920F920FB60F921124F8
:105040002F933F938F939F93AF93BF938091CD07FF
:105050009091CE07A091CF07B091D0073091CC07A7
:1050600023E0230F2D3720F40196A11DB11D05C0AB
:1050700026E8230F0296A11DB11D2093CC07809333
:10508000CD079093CE07A093CF07B093D007809120
:10509000D1079091D207A091D307B091D407019680
:1050A000A11DB11D8093D1079093D207A093D30780
:1050B000B093D407BF91AF919F918F913F912F9162
:1050C0000F900FBE0F901F9018953FB7F8948091E6
:1050D000D1079091D207A091D307B091D40726B5FC
:1050E000A89B05C02F3F19F00196A11DB11D3FBF20
:1050F0006627782F892F9A2F620F711D811D911DB0
:1051000042E0660F771F881F991F4A95D1F70895CF
:105110008F929F92AF92BF92CF92DF92EF92FF92C7
:105120006B017C010E9465284B015C01C114D10414
:10513000E104F104F1F00E94262C0E946528681910
:1051400079098A099B09683E73408105910570F3CE
:1051500021E0C21AD108E108F10888EE880E83E048
:10516000981EA11CB11CC114D104E104F10429F75B
:10517000DDCFFF90EF90DF90CF90BF90AF909F90EA
:105180008F9008958230910538F0880F991F880F0D
:10519000991F05970197F1F70895789484B5826077
:1051A00084BD84B5816084BD85B5826085BD85B5CB
:1051B000816085BDEEE6F0E0808181608083E1E87A
:1051C000F0E01082808182608083808181608083B2
:1051D000E0E8F0E0808181608083E1EBF0E08081B5
:1051E00084608083E0EBF0E0808181608083EAE787
:1051F000F0E0808184608083808182608083808110
:10520000816080838081806880831092C1000895CE
:105210008E3008F08E5087702091320590E4299FDF
:1052200090011124822B80937C0080917A0080640D
:1052300080937A0080917A0086FDFCCF809178007F
:105240002091790090E0922B0895833081F028F42A
:10525000813099F08230A1F008958730A9F088302C
:10526000B9F08430D1F4809180008F7D03C08091AB
:1052700080008F7780938000089584B58F7702C077
:1052800084B58F7D84BD08958091B0008F7703C071
:105290008091B0008F7D8093B0000895CF93DF930D
:1052A00090E0FC01EC57FF4E2491FC01E856FF4EC4
:1052B0008491882349F190E0880F991FFC01E05404
:1052C000FF4EA591B4918A549F4EFC01C591D49193
:1052D0009FB7611108C0F8948C91209582238C931C
:1052E000888182230AC0623051F4F8948C91322F65
:1052F000309583238C938881822B888304C0F89413
:105300008C91822B8C939FBFDF91CF9108950F9347
:105310001F93CF93DF931F92CDB7DEB7282F30E0D6
:10532000F901E059FF4E8491F901EC57FF4E1491B9
:10533000F901E856FF4E04910023C9F0882321F0BB
:1053400069830E9425296981E02FF0E0EE0FFF1F9D
:10535000EA54FF4EA591B4919FB7F8948C916111D6
:1053600003C01095812301C0812B8C939FBF0F90A8
:10537000DF91CF911F910F910895CF93DF93282F45
:1053800030E0F901E059FF4E8491F901EC57FF4EEE
:10539000D491F901E856FF4EC491CC2391F08111CC
:1053A0000E942529EC2FF0E0EE0FFF1FE455FF4E81
:1053B000A591B4912C912D2381E090E021F480E01F
:1053C00002C080E090E0DF91CF910895CF92DF920C
:1053D000EF92FF920F931F93CF93DF937C016A01AB
:1053E000EB0100E010E00C151D0571F06991D7018B
:1053F000ED91FC910190F081E02DC7010995892B79
:1054000019F00F5F1F4FEFCFC801DF91CF911F91B0
:105410000F91FF90EF90DF90CF9008956115710587
:1054200081F0DB010D900020E9F7AD0141505109F9
:10543000461B570BDC01ED91FC910280F381E02DBE
:10544000099480E090E008950C940E2ADC01ED911F
:10545000FC910190F081E02D09948F929F92AF9280
:10546000BF92DF92EF92FF920F931F93CF93DF9340
:10547000CDB7DEB7A1970FB6F894DEBF0FBECDBF94
:105480007C01F42FD52ECB0119A2223008F42AE09A
:105490008E010F5D1F4F822E912CA12CB12C6F2FEE
:1054A0007D2DA50194010E94562EF22FD32ECA0104
:1054B000015011096A3014F4E0E301C0E7E3E60F9C
:1054C000D801EC93232B242B252B49F7B801C701D6
:1054D0000E940E2AA1960FB6F894DEBF0FBECDBF74
:1054E000DF91CF911F910F91FF90EF90DF90BF90D0
:1054F000AF909F908F900895CF92DF92EF92FF929E
:105500000F931F93CF93DF93EC016A017B01211569
:10551000310579F4E881F9810190F081E02D642F63
:10552000DF91CF911F910F91FF90EF90DF90CF907F
:1055300009942A303105E9F477FF1AC06DE20E9420
:10554000262A8C0144275527BA014C195D096E099A
:105550007F092AE0CE010E942D2A800F911FDF9142
:10556000CF911F910F91FF90EF90DF90CF90089512
:105570002AE0B701A601CE01DF91CF911F910F91D3
:10558000FF90EF90DF90CF900C942D2A21153105DC
:1055900041F4DC01ED91FC910190F081E02D642F4C
:1055A00009940C942D2A9A01462F50E060E070E097
:1055B0000C94C62A9A01AB0160E070E00C94C62AF4
:1055C0004F925F926F927F928F929F92AF92BF9213
:1055D000CF92DF92EF92FF920F931F93CF93DF93BF
:1055E000EC016A017B01B22E9A01AB01C701B60141
:1055F0000E94422E882319F06EE876E027C026012B
:105600003701E89477F82FEF3FEF4FE75FE7C301EB
:10561000B2010E94422E81110DC02FEF3FEF4FE7E4
:105620005FE7C301B2010E948C2C18161CF462E9DA
:1056300076E00CC02FEF3FEF4FE75FE4C701B60104
:105640000E94DB2D1816ACF466E976E0CE01DF91FE
:10565000CF911F910F91FF90EF90DF90CF90BF906F
:10566000AF909F908F907F906F905F904F900C9431
:105670000E2A2FEF3FEF4FE75FECC701B6010E9404
:105680008C2C87FDE1CF20E030E0A901C701B601F5
:105690000E948C2C87FF0AC06DE2CE010E94262A50
:1056A0008C01F7FAF094F7F8F09402C000E010E0F3
:1056B000A12C60E070E080E09FE3AB1441F020E0BB
:1056C00030E040E251E40E94902CA394F6CF9B017D
:1056D000AC01C701B6010E94282C6B017C010E941D
:1056E000FD2C2B013C010E94292D9B01AC01C7011F
:1056F000B6010E94272C6B017C012AE0B301A201B4
:10570000CE010E942D2A080F191FBB2039F06AE92B
:1057100076E0CE010E940E2A080F191F7B2C7720FD
:1057200041F120E030E040E251E4C701B6010E94BF
:10573000DF2D6B017C010E94F82C4B01AA2497FC01
:10574000A094BA2C2AE030E0B501A401CE010E9459
:105750007C2A080F191FC501B4010E942B2D9B0143
:10576000AC01C701B6010E94272C6B017C017A9421
:10577000D6CFC801DF91CF911F910F91FF90EF908D
:10578000DF90CF90BF90AF909F908F907F906F9061
:105790005F904F9008950C94E02A4F925F926F9221
:1057A0007F92AF92BF92CF92DF92EF92FF920F93D0
:1057B0001F93CF93DF93CDB7DEB729013A01621B68
:1057C000730B840B950B29893A894B895C892A19BB
:1057D0003B094C095D09298B3A8B4B8B5C8B9B01F8
:1057E000AC0169897A898B899C890E94462EE418CC
:1057F000F50806091709A80197010E94782E2A0DBD
:105800003B1D4C1D5D1DCA01B901DF91CF911F9158
:105810000F91FF90EF90DF90CF90BF90AF907F906F
:105820006F905F904F9008950E94B72E08950E9448
:10583000CD280E94162C0E94E413C0E0D0E00E9404
:1058400043182097E1F30E940000F9CF08955058C3
:10585000BB27AA270ED075C166D130F06BD120F0DE
:1058600031F49F3F11F41EF45BC10EF4E095E7FBA9
:1058700051C1E92F77D180F3BA1762077307840704
:10588000950718F071F49EF58FC10EF4E0950B2E7C
:10589000BA2FA02D0B01B90190010C01CA01A00182
:1058A0001124FF27591B99F0593F50F4503E68F1DD
:1058B0001A16F040A22F232F342F4427585FF3CF1E
:1058C000469537952795A795F0405395C9F77EF4EF
:1058D0001F16BA0B620B730B840BBAF09150A1F038
:1058E000FF0FBB1F661F771F881FC2F70EC0BA0FBE
:1058F000621F731F841F48F4879577956795B79546
:10590000F7959E3F08F0B3CF9395880F08F099273D
:10591000EE0F979587950895D9D008F481E0089502
:105920000CD00FC107D140F0FED030F021F45F3F22
:1059300019F0F0C0511139C1F3C014D198F3992373
:10594000C9F35523B1F3951B550BBB27AA27621743
:105950007307840738F09F5F5F4F220F331F441F88
:10596000AA1FA9F333D00E2E3AF0E0E830D09150C0
:105970005040E695001CCAF729D0FE2F27D0660FAD
:10598000771F881FBB1F261737074807AB07B0E8EC
:1059900009F0BB0B802DBF01FF2793585F4F2AF002
:1059A0009E3F510568F0B6C000C15F3FECF3983EE2
:1059B000DCF3869577956795B795F7959F5FC9F75F
:1059C000880F911D9695879597F90895E1E0660FE8
:1059D000771F881FBB1F621773078407BA0720F061
:1059E000621B730B840BBA0BEE1F88F7E0950895CA
:1059F00004D06894B111D9C00895BCD088F09F57E5
:105A000090F0B92F9927B751A0F0D1F0660F771F0A
:105A1000881F991F1AF0BA95C9F712C0B13081F0EA
:105A2000C3D0B1E00895C0C0672F782F8827B85F32
:105A300039F0B93FCCF3869577956795B395D9F74B
:105A40003EF490958095709561957F4F8F4F9F4F55
:105A50000895E89409C097FB3EF490958095709561
:105A600061957F4F8F4F9F4F9923A9F0F92F96E9AA
:105A7000BB279395F695879577956795B795F1111F
:105A8000F8CFFAF4BB0F11F460FF1BC06F5F7F4FBC
:105A90008F4F9F4F16C0882311F096E911C07723CE
:105AA00021F09EE8872F762F05C0662371F096E8D7
:105AB000862F70E060E02AF09A95660F771F881FA6
:105AC000DAF7880F9695879597F90895990F00084A
:105AD000550FAA0BE0E8FEEF16161706E807F907C0
:105AE000C0F012161306E407F50798F0621B730B5B
:105AF000840B950B39F40A2661F0232B242B252BDC
:105B000021F408950A2609F4A140A6958FEF811D7E
:105B1000811D089597F99F6780E870E060E008951F
:105B20009FEF80EC089500240A94161617061806B5
:105B30000906089500240A94121613061406050691
:105B40000895092E0394000C11F4882352F0BB0F22
:105B500040F4BF2B11F460FF04C06F5F7F4F8F4F85
:105B60009F4F089557FD9058440F551F59F05F3FC0
:105B700071F04795880F97FB991F61F09F3F79F06F
:105B800087950895121613061406551FF2CF4695F1
:105B9000F1DF08C0161617061806991FF1CF869573
:105BA0007105610508940895E894BB276627772757
:105BB000CB0197F908958ADF08F48FEF08950BD091
:105BC000C0CFB1DF28F0B6DF18F0952309F0A2CFDF
:105BD000A7CF1124EACFC6DFA0F3959FD1F3950F8D
:105BE00050E0551F629FF001729FBB27F00DB11D61
:105BF000639FAA27F00DB11DAA1F649F6627B00DF1
:105C0000A11D661F829F2227B00DA11D621F739FD9
:105C1000B00DA11D621F839FA00D611D221F749FE7
:105C20003327A00D611D231F849F600D211D822F2E
:105C3000762F6A2F11249F5750408AF0E1F0882375
:105C40004AF0EE0FFF1FBB1F661F771F881F915082
:105C50005040A9F79E3F510570F05CCFA6CF5F3F43
:105C6000ECF3983EDCF3869577956795B795F795B5
:105C7000E7959F5FC1F7FE2B880F911D969587953D
:105C800097F9089523DF880B990B0895DB018F9313
:105C90009F930E94972EBF91AF91A29F800D911D5F
:105CA000A39F900DB29F900D11240895A1E21A2E8A
:105CB000AA1BBB1BFD010DC0AA1FBB1FEE1FFF1FB0
:105CC000A217B307E407F50720F0A21BB30BE40B00
:105CD000F50B661F771F881F991F1A9469F7609547
:105CE0007095809590959B01AC01BD01CF01089501
:105CF000052E97FB1EF400940E948F2E57FD07D0AF
:105D00000E94562E07FC03D04EF40C948F2E509513
:105D10004095309521953F4F4F4F5F4F0895909597
:105D20008095709561957F4F8F4F9F4F08950E948A
:105D3000A82EA59F900DB49F900DA49F800D911D3E
:105D400011240895EE0FFF1F0590F491E02D0994A2
:105D5000A29FB001B39FC001A39F700D811D1124AC
:105D6000911DB29F700D811D1124911D089581E038
:105D700090E0F8940C94D22EF999FECF92BD81BD9B
:105D8000F89A992780B50895262FF999FECF1FBA62
:105D900092BD81BD20BD0FB6F894FA9AF99A0FBE54
:085DA00001960895F894FFCF6D
:105DA8000000D5078000010000001801010104016E
:105DB800000096430000A042000096430000A04265
:105DC8000A0A000103070F1F3F7F0080C0E0F0F8B8
:105DD800FCFE0000000000000000000000000000C1
:105DE80000000000000000000000000000000000AB
:105DF800000000000000000000000000000000009B
:105E0800000000000000000000000000000000008A
:105E180000808080000000000000000000000000FA
:105E28000000008080C0C0000000000000000000EA
:105E3800000000000000000000000000000000005A
:105E4800000000000000000000000000000000004A
:105E5800000000000000000000000000000000003A
:105E680000000000000080C0E0F0F8FCF8E000004E
:105E7800000000000000000000000000000000809A
:105E8800808080800080800000000080808080808A
:105E980000FFFFFF000000008080808000008080FD
:105EA800000080FFFF80800080800080808080006C
:105EB80080800000000000808000008C8E8400003C
:105EC80080F8F8F8800000000000000000000000E2
:105ED8000000F0F0F0F0F0F0F0F0F0F0F0F0E0E0BA
:105EE800C08000E0FCFEFFFFFF7FFFFFFFFFFF0019
:105EF80000000000000000000000000000FEFFC7D6
:105F08000101010183FFFF00007CFEC701010101BF
:105F180083FFFFFF0038FEC78301010183C7FFFF2E
:105F2800000001FFFF010100FFFF07010101000060
:105F38007FFF80000000FFFF7F0000FFFFFF0000E1
:105F480001FFFFFF0100000000000000000000004A
:105F58000000030F3F7F7FFFFFFFFFFFFFFFE7C743
:105F6800C78F8F9FBFFFFFC3C0F0FFFFFFFFFFFC7E
:105F7800FCFCFCFCFCFCFCF8F8F0F0E0C0000103C1
:105F880003030303010303000000000103030303E9
:105F980001010301000000010303030301010303DE
:105FA80000000003030000000303000000000000DD
:105FB80000010303030303010000000103010000C3
:105FC80000030301000000000000000000000000C2
:105FD800000000000080C0E0F0F9FFFFFFFFFF3F76
:105FE8001F0F87C7F7FFFF1F1F3DFCF8F8F8F87C65
:105FF8007DFFFFFFFFFFFFFFFF7F3F0F07003030F0
:106008000000000000000000000000000000000088
:10601800000000000000FEFEFC0000000000000080
:10602800000000000000000000000000000000E088
:10603800C000000000000000000000003030000038
:106048000000000000000000000000000000000048
:10605800000000C0FEFFFFFFFFFFFFFFFFFF7F7F85
:106068003F1F0F071F7FFFFFF8F8FFFFFFFFFFFE2F
:10607800F8E0000000010000000000000000FEFE43
:10608800000000FCFEFC0C06060EFCF80000F0F810
:106098001C0E0606060CFFFFFF0000FEFE000000B7
:1060A80000FCFEFC00183C7E66E6CE84000006FF7D
:1060B800FF0606FCFEFC0C0606060000FEFE0000BD
:1060C800C0F8FC4E4646464E7C7840183C76E6CEF4
:1060D800CC8000000000000000000000000000006C
:1060E80000000000000001070F1F1F3F3F3F3F1F38
:1060F8000F030000000000000000000000000F0F68
:106108000000000F0F0F000000000F0F0000030732
:106118000E0C18180C060F0F0F0000010F0E0C18AC
:106128000C0F070100040E0C180C0F070000000FDD
:106138000F00000F0F0F0000000000000F0F0000FD
:106148000007070C0C181C0C060600040E0C180C93
:106158000F07000000000000000000000000000021
:106168000000000000000000000000000000000027
:106178000000000000000000000000000000000017
:106188000000000000000000000000000000000007
:1061980000000000000000000000000000000000F7
:1061A80000000000000000000000000000000000E7
:1061B80000000000000000000000000000000000D7
:1061C80000000000000000000000000000000000C7
:1061D8000000015258204F4E2031003C3C3C3C000E
:1061E8005258204F4E2032003E3E3E3E0020205561
:1061F800502020200020444F574E202020002042CD
:10620800414E44202B2000204F4B20002042414E7D
:1062180044202D200020534641564F2000204D4554
:106228004E5520004D485A004C4F5720534947209F
:106238002100474F4F442053494720002020202069
:1062480020202020202020204348203C2000203EE1
:1062580000214641562100442F352E3300432F524A
:1062680061636500462F4169727761766500450074
:106278004200410020203C3C205345542046494CD4
:10628800544552203E3E0046494C544552204C4FFE
:10629800570046494C544552204D454449554D00F8
:1062A80046494C54455220484947480020203C3C28
:1062B80020534554204641564F204348203E3E0037
:1062C8004D6164652042792042757A7A20466C795E
:1062D80000205370656369616C206D6164652021DD
:1062E800004241434B204D454E55000000000045FB
:1062F8001A181AED19F519081A171A00000000786B
:1063080021E629142C7F1C851D9C1D361DB21DE716
:106318001D051E000000007821E629DE247F1CA34D
:10632800236B22361DB21DE71D051E0D0A006E6186
:0C6338006E00696E66006F7666002E0035
:00000001FF
